:020000040000FA
:02000000B42822
:080008008428820752345334AE
:10001000323433343234203444346134743461340F
:100020002034733465346E3464346534723420346F
:10003000503449344334203463346F346434653489
:100040002034563431342E34303430342C3420348F
:100050002834433429342034323430343034313489
:10006000203443346F3470347934723469346734F3
:100070006834743420344234793420344634723451
:1000800065346434203448346F34753477346534DF
:100090006C3469346E3467340D340A343C3466345D
:1000A000723465346434403468346F347534773472
:1000B00065346C3469346E3467342E3463346F3491
:1000C0006D342E34613475343E34203468347434E5
:1000D000743470343A342F342F347734773477349F
:1000E0002E3468346F347534773465346C34693445
:1000F0006E3467342E3463346F346D342E3461348F
:1001000075340D340A3400348C00030E8D008312D4
:100110008E0F932812088E008F1891288F140615C1
:1001200093288F1006110B110D0E83008C0E0C0EF0
:100130000900343096009530970000349920A720AC
:100140009920A7209920A7209920A72000341608DD
:10015000940017089500950BAB28940BB028B32892
:1001600017089500AB280034640083161130810015
:1001700005148510061186100612861206178312C2
:1001800085018601061685149920A72021211208D1
:100190008E008F01900191018B168B170021831225
:1001A00021219118D62891148614D82891108610F0
:1001B0000000E5209E209E209E209E209E209E20C6
:1001C0009E209E209E209E20D02812089B006430F6
:1001D0009C0035211A08303E98000B210A309C0003
:1001E00035211A08303E98000B211B08303E98003C
:1001F0000B210D3098000B210A3098000B210800CC
:100200009901190805209800980803190A290B215B
:10021000990A0129080009309300851000000000A8
:100220001C21980C031C1629851417298510930B83
:10023000102985141C2108001E309700970B1E29D9
:1002400008000612000000000000000008309300C3
:100250009201861600000314061F0310920D8612E9
:100260000000930B2929061608009A019C0803191F
:1002700045299B08031945291C089B02031843299B
:0C0280001C089B0745299A0A3929080030
:02400E00FA3F77
:00000001FF
